:100000000428FF3FFF3FFF3F523003138312BD0020
:100010006530BE006130BF006430C0006930C1008F
:100020006E30C2006730C3002030C4004C30C500C1
:100030004D30C6003330C7003330C8003530C900FA
:100040002E30CA002E30CB002E30CC00CD015430E3
:10005000CE002030CF003D30D0002030D100D20182
:100060005430D3002030D4003D30D5002030D600AD
:10007000D7010317831689010D30880003138312FB
:100080008501870186011D3083168500CF308600EB
:10009000F030870007308312DC000330DD000230CF
:1000A000DE000130DF00E0010530E1000730E20052
:1000B0000130E3000630E40079210C30EA0003242B
:1000C0000130EA0003240130DC000130DD003D3066
:1000D000DE0059260230DC000130DD004E30DE004B
:1000E00059260230DC000930DD00DF30DE009E26BC
:1000F0000230DC000A30DD004330DE009E26803016
:1001000083169F00413083129F00AB01AC01AD010B
:10011000AE01AF010A302F020318D0284130FB0096
:10012000FF30FA00FB0B95289828FA0B95289228A7
:10013000C330FA00FA0B9A2800009F1400309F1871
:100140000130F4007408013A03199E281E08B0001B
:10015000B1013008F100F0017008B0007108B10081
:1001600083161E08F0070318F10A70088312B00006
:100170007108B1008A151D208A112B08F4002C0883
:10018000F5002D08F6002E08F700BD227008AB0020
:100190007108AC007208AD007308AE00AF0A8A287F
:1001A0002B08F0002C08F1002D08F2002E08F300B7
:1001B0000030F4000030F5002030F6008130F70008
:1001C0007C240030F400C030F5007F30F600883029
:1001D000F7005F237008AB007108AC007208AD0037
:1001E0007308AE000030F4000030F5004830F6002F
:1001F0008530F7007C240030F400B830F5002A3058
:10020000F6008A30F7008A156B208A117008AB005F
:100210007108AC007208AD007308AE004725700885
:10022000DA007108DB000A30F4000030F5005A08EB
:10023000F0005B08F1008A1500208A117008D800D0
:100240007108D9005808B2005908B3000A30F40008
:100250000030F5005A08F0005B08F1008A15002014
:100260008A117808F0007908F1007008B40071086C
:10027000B5005808DC005908DD003630DE000126E4
:100280000230DC000130DD003630DE0059262C3033
:10029000E5008A1560208A113408303FE5008A1590
:1002A00060208A110230DC000130DD005330DE00B6
:1002B00059260630FC00FF30FB00FF30FA00FC0B33
:1002C00062296929FB0B65296829FA0B65296229CE
:1002D0005F291A30FB00FF30FA00FB0B70297329ED
:1002E000FA0B70296D294230FA00FA0B752985281E
:1002F00078290C270C270C275D08F0000130F70047
:10030000700803198729F70D7710FF3F81297708B7
:10031000A5005E08F0000130F1007008031994296F
:10032000F10D7110FF3F8E297108A6005F08F000E3
:100330000130F60070080319A129F60D7610FF3F71
:100340009B297608A7006008F0000130F5007008CE
:100350000319AE29F50D7510FF3FA8297508A800EF
:100360006208F0000130F40070080319BB29F40D95
:100370007410FF3FB5297408A3006308F000013032
:10038000F30070080319C829F30D7310FF3FC22949
:100390007308AA006408F0000130F2007008031925
:1003A000D529F20D7210FF3FCF297208A2005C0818
:1003B000A4006108A1005C08840071087704F000C3
:1003C0007608F00475087004F1007109F0007008F7
:1003D000800584177108F000F00970088005610835
:1003E000840073087404F0007208F004F0097008C7
:1003F00080058417700880055C0884007508760401
:10040000F0007008800461088400720880048A1576
:1004100087208A112209F000700880050C27220825
:1004200080048A1587208A112209F000700880054F
:100430000C27220880048A1587208A112209F000DF
:10044000700880050C2724088400270880042809E8
:10045000F0007008800521088400220880048A15B5
:1004600087208A112209F000700880050C272208D5
:1004700080048A1587208A112209F00070088005FF
:10048000240884002709F0007008800525088004EE
:1004900021088400220880048A1587208A112209F5
:1004A000F000700880050C27240884002509F0005E
:1004B0007008800528088004210884002208800430
:1004C0008A1587208A112209F00070088005240807
:1004D00084002809F00070088005210884002208A3
:1004E00080048A1587208A112209F000700880058F
:1004F0000C27220880048A1587208A112209F0001F
:1005000070088005240884002808800421088400DD
:10051000220880048A1587208A112209F0007008B9
:1005200080050C27240884002809F0007008800545
:1005300021088400220880048A1587208A11220954
:10054000F000700880052408840027082804F000C3
:100550002608F0042508F0047008800421088400AF
:10056000220880048A1587208A112209F000700869
:1005700080050C270130A9000800031383127208BC
:100580007606A000F801F90173087702031CE02A3F
:100590007708FD007308F7007D08F3007608FD007A
:1005A0007208F6007D08F2007508FD007108F5007C
:1005B0007D08F1007408FD007008F4007D08F0006B
:1005C000770803195B2B7208FA00F217F617770801
:1005D0007302F7000319132B08307702031C092B51
:1005E000F7007408F9007508F4007608F500F601C4
:1005F00008307702031C092BF7007408F90075080E
:10060000F400F50108307702031C092B7A08F20088
:100610005B2B77080319132B0310F60CF50CF40C65
:10062000F90CF70B0C2BA01F202BF909F409F50985
:10063000F609F90A0319F40A0319F50A0319F60A67
:100640007908F80774080318740FF0077508031881
:10065000750FF10776080318760FF207A01B392BE8
:10066000031C492BF20CF10CF00CF80CF30F492B86
:10067000552B03184D2BF809F009F109F209F80A76
:100680000319F00A0319F10A0319F20A8030FA0675
:10069000512B0130FC00E3245D2B0230FC00E324ED
:1006A0005D2B0430FC00D5265D2B0830FC008A153C
:1006B00044208A115D2B0030FC0000000800031369
:1006C000831277080319EE2B73080319F32B7208B2
:1006D00076068039FA00F217F617A0017208F800C2
:1006E0007108FC007008FD007408FD027508031C09
:1006F000750FFC027608031C760FF802F801FC0166
:10070000FD01031C8A2B0310F20CF10CF00CF80C09
:100710000130A0007708F302031C942B7E302007E1
:10072000F3070318F82B992B7E302007F307031CDF
:10073000FD2B1830FA07FD0DFC0DF80DF00DF10D35
:10074000F20DA00D7408F0027508031C750FF1027C
:100750007608031C760FF202760DA004201CB22B43
:100760007D14BD2B7408F00775080318750FF10789
:1007700076080318760AF2077D10FA031F307A050F
:10078000031D9B2B7B1B7D1CE42B0310F00DF10D37
:10079000F20DA00D7408F0027508031C750FF1022C
:1007A0007608031C760FF202760D20040139FD074E
:1007B0000318FC0A0319F80A031DE42BF80CFC0CBF
:1007C000FD0CF30A0319F82BFA1FF8137808F2004E
:1007D0007C08F1007D08F0000030012C01308A1502
:1007E00082208A11012C02308A1573208A11012C73
:1007F00004308A1544208A11012C08308A155220B1
:100800008A110000080003138312210884002209C2
:10081000F000700880052309F000700880052408A6
:10082000840026082504F0002708F0042808F004B6
:10083000F00970088005EA1F1F2C250880046A1F34
:10084000232C26088004EA1E272C270880046A1E11
:100850002B2C280880042108840029080319352C32
:100860002309F00070088005372C23088004220833
:1008700080048A1587208A112209F00070088005FB
:100880002309F00070088005240884002608250448
:10089000F0002708F0042808F004F009700880052B
:1008A000EA1D542C250880046A1D582C2608800453
:1008B000EA1C5C2C270880046A1C602C2808800431
:1008C00021088400290803196A2C2309F000700804
:1008D00080056C2C23088004220880048A15872058
:1008E0008A112209F00070088005290803197A2C62
:1008F0000C277B2C1D27080003138312FB017308B0
:10090000031D77080319D32C72087606FA007708BE
:10091000F3077E30031C902CF3020318D82C932C81
:10092000F302031CDD2C7208F8007108FC0070084B
:10093000FD00F817F6170310F201F101F00118306D
:10094000A0007D1CAD2C7408F00775080318750F06
:10095000F10776080318760FF207F20CF10CF00C91
:10096000F80CFC0CFD0C0310A00BA12CF21BBD2CF1
:10097000F80DF00DF10DF20DF3037B1B701CCF2C65
:10098000F81FCF2CF00A0319F10A0319F20A031D0C
:10099000CF2CF20CF10CF00CF30A0319D82CFA1F2F
:1009A000F2130030E12C01308A1573208A11E12CFA
:1009B00002308A1544208A11E12C04308A15522015
:1009C0008A1100000800031383127C181B2DFC18E9
:1009D000EC2C7C19402DE52CA0017208031D0C2D78
:1009E0007108F2007008F1007808F000F801A01515
:1009F0007208031D0C2D7108F2007008F100F0015F
:100A0000A01120167208031D0C2D7108F200F101CF
:100A1000A015720803192E2D2008F302031D031CD4
:100A2000342D0310F21B1B2DF80DF00DF10DF20DFE
:100A3000F30B122D342D7B1B701C3A2DF81F3A2D11
:100A4000F00A0319F10A0319F20A031D3A2DF20CF8
:100A5000F10CF00CF30A0319402D3A2D0130FC0083
:100A60008A1573208A11452D0230FC008A15522008
:100A70008A11452D0430FC008A157C208A11452DF1
:100A80000830FC008A1544208A1100000800031376
:100A90008312FB01FC01FA0173080319862DF2177A
:100AA0008E30F302F31B572D0319572D892DF309AF
:100AB000F30A08307302031C6C2DF300F10D720869
:100AC000F100F20108307302031C6C2DF10DF101ED
:100AD0007308031D0310742D73080319742D03107C
:100AE000F20CF10CF30B6F2D7B1B711C7E2D031C84
:100AF0007E2DF10A0319F20AF21B952DFA1F982D8B
:100B0000F209F109F10A0319F20A982DF201F10133
:100B1000982D7B14FB1F9B2DF201FA1F9B2DFF309C
:100B2000F200F100FA0DF20C9B2D0130FC009D2D1E
:100B30000030FC009D2DFF30FC00FC080319A32DA4
:100B40008A1535208A117108F0007208F10008003A
:100B5000031383126708840020308000670AF000C6
:100B6000700884002030800002306707F0007008B1
:100B700084002030800003306707F0007008840094
:100B80002030800004306707F000700884003030A7
:100B9000800005306707F000700884008001043091
:100BA000E8006608003C031DD72D6508003C0318CB
:100BB000002E68086707E9000A30F400F5016508AF
:100BC000F0006608F1008A1500208A117808F0000C
:100BD0007908F1003030F00769088400700880005F
:100BE0000A30F400F5016508F0006608F1008A1586
:100BF00000208A117008E5007108E600E803D12D95
:100C0000080003138312E0015C08E1005D08E200C4
:100C100080305D06F00080307002031D112E003020
:100C20005C0203181D2E0130E0005C08003CE1006E
:100C30005D08031C013FE201E2026108E500620871
:100C4000E6005E08E700A8250630DF005F08003CEC
:100C500003183E2E5F085E07F20001305F02F000CD
:100C6000F101031CF10370085E0784000008F00026
:100C70007208840070088000DF03262E5E0884005E
:100C80002030800060080319582E5F085E0784003A
:100C90000008F2007208203A031D502EDF0A452E8C
:100CA000DF035F085E07F000700884002D308000CD
:100CB00008006B2E803003138312DC007E2EC030C0
:100CC000DC007E2E9430DC007E2ED430DC007E2EC4
:100CD0008030DC007E2E031383125C08013A031976
:100CE0005A2E5C08023A03195F2E5C08033A031976
:100CF000622E5C08043A0319652E682E5D03F0002D
:100D00005C08F0077008DC007008EA000324A90101
:100D1000DF015F085E0784000008F0007008031917
:100D20009B2E5F085E0784000008E5008A1560209E
:100D30008A11DF0A892E0130A9000800B02E803008
:100D400003138312DC00C32EC030DC00C32E9430AA
:100D5000DC00C32ED430DC00C32E8030DC00C32E78
:100D6000031383125C08013A03199F2E5C08023AB0
:100D70000319A42E5C08033A0319A72E5C08043A51
:100D80000319AA2EAD2E5D03F0005C08F007700871
:100D9000DC000130A9007008EA000324A9015E0804
:100DA000EA0003240130A900080003138312A00104
:100DB0007208031DEC2E7108F2007008F100F001BA
:100DC000A0157208031DEC2E7108F200F101A011AC
:100DD000201672080319FA2E2008F302031D031CC3
:100DE000002F0310F21B062FF00DF10DF20DF30B87
:100DF000F22E002F0130FC008A1573208A110B2F70
:100E00000230FC008A1552208A110B2F0430FC009E
:100E10008A157C208A110800083003138312FB0016
:100E2000FF30FA00FB0B152F182FFA0B152F122F7E
:100E30001E30FA00FA0B1A2F080010300313831229
:100E4000FA00FA0B212F00000800FF3FFF3FFF3F91
:100E5000FF3FFF3FFF3FFF3FFF3FFF3FFF3FFF3FA2
:100E6000FF3FFF3FFF3FFF3FFF3FFF3FFF3FFF3F92
:100E7000FF3FFF3FFF3FFF3FFF3FFF3FFF3FFF3F82
:100E8000FF3FFF3FFF3FFF3FFF3FFF3FFF3FFF3F72
:100E9000FF3FFF3FFF3FFF3FFF3FFF3FFF3FFF3F62
:100EA000FF3FFF3FFF3FFF3FFF3FFF3FFF3FFF3F52
:100EB000FF3FFF3FFF3FFF3FFF3FFF3FFF3FFF3F42
:100EC000FF3FFF3FFF3FFF3FFF3FFF3FFF3FFF3F32
:100ED000FF3FFF3FFF3FFF3FFF3FFF3FFF3FFF3F22
:100EE000FF3FFF3FFF3FFF3FFF3FFF3FFF3FFF3F12
:100EF000FF3FFF3FFF3FFF3FFF3FFF3FFF3FFF3F02
:100F0000FF3FFF3FFF3FFF3FFF3FFF3FFF3FFF3FF1
:100F1000FF3FFF3FFF3FFF3FFF3FFF3FFF3FFF3FE1
:100F2000FF3FFF3FFF3FFF3FFF3FFF3FFF3FFF3FD1
:100F3000FF3FFF3FFF3FFF3FFF3FFF3FFF3FFF3FC1
:100F4000FF3FFF3FFF3FFF3FFF3FFF3FFF3FFF3FB1
:100F5000FF3FFF3FFF3FFF3FFF3FFF3FFF3FFF3FA1
:100F6000FF3FFF3FFF3FFF3FFF3FFF3FFF3FFF3F91
:100F7000FF3FFF3FFF3FFF3FFF3FFF3FFF3FFF3F81
:100F8000FF3FFF3FFF3FFF3FFF3FFF3FFF3FFF3F71
:100F9000FF3FFF3FFF3FFF3FFF3FFF3FFF3FFF3F61
:100FA000FF3FFF3FFF3FFF3FFF3FFF3FFF3FFF3F51
:100FB000FF3FFF3FFF3FFF3FFF3FFF3FFF3FFF3F41
:100FC000FF3FFF3FFF3FFF3FFF3FFF3FFF3FFF3F31
:100FD000FF3FFF3FFF3FFF3FFF3FFF3FFF3FFF3F21
:100FE000FF3FFF3FFF3FFF3FFF3FFF3FFF3FFF3F11
:100FF000FF3FFF3FFF3FFF3FFF3FFF3FFF3FFF3F01
:1010000003138312F801F9011030FC00710DF80D83
:10101000F90D7408F8027508031C750FF90203181E
:1010200018287408F80775080318750FF9070310D6
:10103000F00DF10DFC0B0628080003138312700855
:10104000F8007108F000F101F201F301FB01FC016D
:101050009630F300FA017008F1007808F000F8010A
:10106000F2018A11D5268A150800031383127B1416
:10107000FB1F4228F201FA1FFF30F200F100F000DE
:10108000FA0DF20CFF30080003138312FB14FB1F50
:101090005028FF30F300F200F100F000FA0DF20CDE
:1010A000FF300800031383127B15FB1F5E280130FD
:1010B000F300F201F101F001FA0DF20CFF3008002B
:1010C00003138312A9016508EA008A1103248A1513
:1010D0000130A9000800031383128030F6068A113C
:1010E000BD228A15080003138312F201F101F001F9
:1010F000F801F3010030080003138312FA1FF21302
:101100000030080003138312FB15FF3008000000B5
:101110000800FF3FFF3FFF3FFF3FFF3FFF3FFF3F15
:04400E00E420FF3F6C
:00000001FF
